:020000040800F2
:10000000D88B0020690200083D280008FF24000862
:1000100039280008A5050008153000080000000078
:10002000000000000000000000000000432800085D
:1000300013070008000000004128000845280008B8
:10004000830200088302000883020008830200087C
:10005000830200088302000883020008830200086C
:10006000830200088302000883020008830200085C
:1000700083020008A905000883020008B9050008EA
:10008000C9050008D905000883020008830200089A
:10009000830200088302000883020008830200082C
:1000A000830200088302000883020008830200081C
:1000B000830200088302000883020008830200080C
:1000C00083020008830200088302000883020008FC
:1000D00083020008F52F000805300008830200089D
:1000E00083020008830200088302000883020008DC
:1000F00083020008830200088302000883020008CC
:1001000083020008830200088302000883020008BB
:1001100045290008830200088302000883020008C2
:100120008302000883020008E90500088302000832
:10013000830200088302000883020008830200088B
:10014000830200088302000883020008830200087B
:100150008302000883020008F905000883020008F2
:10016000830200088302000883020008830200085B
:1001700083020008830200088302000800000000D8
:10018000830200088302000800F002F800F05CF827
:100190000AA090E8000C82448344AAF10107DA45E2
:1001A00001D100F051F8AFF2090EBAE80F0013F0D8
:1001B000010F18BFFB1A43F001031847B8370000BE
:1001C000D83700000A444FF0000C10F8013B13F040
:1001D000070408BF10F8014B1D1108BF10F8015BA0
:1001E000641E05D010F8016B641E01F8016BF9D193
:1001F00013F0080F1EBF10F8014BAD1C0C1B09D1EA
:100200006D1E58BF01F801CBFAD505E014F8016B5B
:1002100001F8016B6D1EF9D59142D6D370470000ED
:100220000023002400250026103A28BF78C1FBD8FF
:10023000520728BF30C148BF0B6070471FB503F09D
:100240005BFB1FBD10B510BD00F072F91146FFF742
:10025000F5FF03F079FA00F090F903B4FFF7F2FF2D
:1002600003BC00F099F9000009488047094800479D
:10027000FEE7FEE7FEE7FEE7FEE7FEE7FEE7FEE756
:10028000FEE7FEE704480549054A064B70470000B3
:100290003129000889010008D87B0020D88B002074
:1002A000D8830020D883002053EA020C00F0698034
:1002B0002DE9F04B4FF00006002B1FBFB3FA83F57A
:1002C00003FA05F424FA05F65E4012BF1643B2FAAB
:1002D00082F502FA05F4C5F120051EBF22FA05FCDD
:1002E00044EA0C04203556EA044C4FEA144418BF83
:1002F000641C4FF000084FF00009904271EB030CB2
:1003000039D3002919BFB1FA81F701FA07F6B0FA1B
:1003100080F700FA07F6C7F120071EBF20FA07FC96
:1003200046EA0C062037B6FBF4FCA7EB0507103FA6
:1003300007F01F0BCBF120060CFA0BFB2CFA06F68C
:1003400044BFB3460026202FA4BF5E464FF0000BEB
:100350005BEA060C08BF4FF0010B19EB0B09ABFB76
:10036000027C48EB0608C01B06FB02CC0BFB03CC4F
:1003700071EB0C01C1E70B46024641464846BDE819
:10038000F08B13B54FF000004FF00001AFF3008089
:10039000BDE81C40704740EA010310B59B070FD130
:1003A000042A0DD310C808C9121F9C42F8D020BAE5
:1003B00019BA884201D9012010BD4FF0FF3010BD9D
:1003C0001AB1D30703D0521C07E0002010BD10F86B
:1003D000013B11F8014B1B1B07D110F8013B11F831
:1003E000014B1B1B01D1921EF1D1184610BD032AEF
:1003F00040F2308010F0030C00F0158011F8013B42
:10040000BCF1020F624498BF11F801CB00F8013B28
:1004100038BF11F8013BA2F1040298BF00F801CBEC
:1004200038BF00F8013B11F0030300F04F80083A99
:10043000C0F0088051F8043B083A51F804CBA0E81A
:100440000810F5E7121D5CBF51F8043B40F8043B6F
:10045000AFF30080D20724BF11F8013B11F801CBA4
:1004600048BF11F8012B24BF00F8013B00F801CB75
:1004700048BF00F8012B70474FF0000200B513464B
:1004800094469646203922BFA0E80C50A0E80C50B4
:10049000B1F12001BFF4F7AF090728BFA0E80C5065
:1004A00048BF0CC05DF804EB890028BF40F8042B5E
:1004B00008BF704748BF20F8022B11F0804F18BFCB
:1004C00000F8012B704770477047704710B5203A0D
:1004D000C0F00B80B1E81850203AA0E81850B1E8FD
:1004E0001850A0E81850BFF4F5AF5FEA027C24BFB3
:1004F000B1E81850A0E8185044BF18C918C0BDE8AA
:1005000010405FEA827C24BF51F8043B40F8043B72
:1005100008BF7047D20728BF31F8023B48BF11F827
:10052000012B28BF20F8023B48BF00F8012B704781
:10053000754600F02BF8AE4605006946534620F09C
:100540000700854618B020B5FFF79CFEBDE82040A7
:100550004FF000064FF000074FF000084FF0000B7F
:1005600021F00701AC46ACE8C009ACE8C009ACE832
:10057000C009ACE8C0098D46704710B50446AFF31A
:1005800000802046BDE81040FFF767BE0048704776
:10059000787B00207047000001491820ABBEFEE7C1
:1005A0002600020000BFFEE710B5024800F078FA0E
:1005B00010BD0000E803002010B5024800F070FAFA
:1005C00010BD00004804002010B5024800F068FA91
:1005D00010BD00006805002010B5024800F060FA68
:1005E00010BD0000C805002010B5024800F058FA00
:1005F00010BD0000A804002010B5024800F050FA19
:1006000010BD0000080500200146087810381823A6
:10061000B0FBF3F20848805CC865032A05D9086876
:100620006FF30900001D886503E008686FF3090097
:100630008865886D70470000023900080146002077
:100640008A6A8B69CBB932B1012A0DD0022A03D054
:10065000032A10D10EE000BFCB6A03F08073B3F120
:10066000807F00D1012007E0CB6AB3F1C07F00D1C9
:10067000012001E000E000BF34E08B69B3F5005FCA
:100680001AD132B1012A07D0022A03D0032A11D18C
:100690000AE000BF01200EE0CB6A03F08073B3F1E3
:1006A000807F00D1012006E0CB6AB3F1C07F00D18A
:1006B000012000E000BF15E032B1012A05D0022A76
:1006C00004D0032A0CD103E000BF00BF012008E0E2
:1006D000CB6A03F08073B3F1807F00D1012000E08A
:1006E00000BF00BF704730B50468246824F480243C
:1006F00005682C60046863608468402C04D1046839
:10070000A2600468E16003E00468A1600468E2603C
:1007100030BD704772B600BFFEE7000010B5002282
:1007200001B909E0012901D10A0205E0022901D13C
:100730000A0201E04FF440720E4B1B6823F4407331
:100740000C4C236023461B681343236023461B681D
:1007500023F0F803236023461B68022444EAC00404
:100760002343044C236023461B6843F480332360F7
:1007700010BD0000103C02401C48006800F40070EE
:10078000B0B11A48006820F400701849086000BF32
:100790000846006840F4006008600846006820F4DD
:1007A0000060086000BF0846006840F40070086000
:1007B0000E48006800F48060B0B10C48006820F476
:1007C00080600A49086000BF0846006840F4805015
:1007D00008600846006820F48050086000BF0846A2
:1007E000006840F48060086070470000003C0240F0
:1007F0000A4A126822F44072084B1A601A461268BC
:1008000042F004021A601A4612684FF4803343EA39
:1008100000231A43014B1A6070470000103C02404D
:10082000074A126822F44072054B1A601A46126891
:100830001A601A46126842F001021A60017070478D
:10084000103C024010B50D49096821F440710B4C71
:1008500021602146096841F4407121602146096800
:1008600041F001012160026000BF00BF00BFBFF383
:100870006F8F00BF00BF00BF436010BD103C02403F
:10088000084A126822F44072064B1A601A4612682F
:1008900042F480721A601A46126842F001021A602D
:1008A00001807047103C0240084A126822F44072EE
:1008B000064B1A601A46126842F400721A601A4611
:1008C000126842F001021A6001607047103C024059
:1008D0002348006800F0100040B12248C06940F091
:1008E00010002049C86110201D4908601C4800689C
:1008F00000F0200040B11B48C06940F008001949D1
:10090000C8612020164908601548006800F04000C2
:1009100040B11448C06940F004001249C861402049
:100920000F4908600E48006800F0800040B10D4893
:10093000C06940F002000B49C86180200849086086
:100940000748006800F0020040B10648C06940F066
:1009500020000449C8610220014908607047000076
:100960000C3C02402806002070B5044600250020FB
:100970001449C86100F058FC054609E0601C38B114
:1009800024B100F051FC401BA04201D9032070BDEE
:100990000D48006800F480300028EFD10A48006854
:1009A00000F0010010B10120074908600648006806
:1009B00000F0F20018B1FFF78BFF0120E7E70020FD
:1009C000E5E70000280600200C3C024070B5044614
:1009D000A56D00F029FC064694F83500022808D0E1
:1009E0008020606500BF002084F8340000BF012033
:1009F00070BD2068006820F016002168086020683B
:100A0000406920F0800021684861206C08B9A06C22
:100A100028B12068006820F008002168086020687C
:100A2000006820F001002168086010E000F0FCFB85
:100A3000801B05280BD920206065032084F8350031
:100A400000BF002084F8340000BF0320D0E72068F6
:100A5000006800F001000028E8D194F85C103F2005
:100A60008840A860012084F8350000BF002084F889
:100A7000340000BF00BFBBE7014691F835000228F3
:100A800003D08020486501207047052081F835009B
:100A90000868006820F001000A6810600020F3E791
:100AA000F8B50446002000908C4800684FF41651B9
:100AB000B0FBF1F7A56D2E6894F85C100820884013
:100AC000304098B12068006800F0040070B12068E0
:100AD000006820F004002168086094F85C10082089
:100AE0008840A860606D40F00100606594F85C107B
:100AF00001208840304068B12068406900F08000E3
:100B000040B194F85C1001208840A860606D40F00E
:100B10000200606594F85C1004208840304068B1A1
:100B20002068006800F0020040B194F85C100420D6
:100B30008840A860606D40F00400606594F85C1027
:100B400010208840304078B32068006800F008002A
:100B500050B394F85C1010208840A86020680068AA
:100B600000F4802080B12068006800F4002028B9DB
:100B7000206CC8B12046216C884715E0A06C98B164
:100B80002046A16C88470FE02068006800F4807060
:100B900028B92068006820F0080021680860206CEF
:100BA00010B12046216C884794F85C1020208840C2
:100BB0003040002865D02068006800F01000002850
:100BC0005FD094F85C1020208840A86094F835002D
:100BD000052828D12068006820F0160021680860E8
:100BE0002068406920F0800021684861206C08B9C5
:100BF000A06C28B12068006820F008002168086017
:100C000094F85C103F208840A860012084F83500EB
:100C100000BF002084F8340000BF206D10B12046D2
:100C2000216D8847F8BD2068006800F4802080B1FD
:100C30002068006800F4002028B9606C10B12046DC
:100C4000616C88471DE0E06BD8B12046E16B8847B6
:100C500017E02068006800F4807068B920680068B8
:100C600020F0100021680860012084F8350000BFE2
:100C7000002084F8340000BFE06B10B12046E16B27
:100C80008847606D38B3606D00F00100F0B1052059
:100C900084F835002068006820F0010021680860B1
:100CA00000BF0098401C0090B84200D905E02068C1
:100CB000006800F001000028F3D100BF012084F893
:100CC000350000BF002084F8340000BFE06C10B194
:100CD0002046E16C884700BFA4E700000C0000201C
:100CE0002DE9F0410446002500F09EFA074614B9AC
:100CF0000120BDE8F081606A00B100BF022084F8E5
:100D0000350000BF002084F8340000BF2068006870
:100D100020F00100216808600AE000F085FAC01B9D
:100D2000052805D920206065032084F83500E0E718
:100D30002068006800F001000028EED120680568F6
:100D400021480540D4E901010843E16808432169CD
:100D5000084361690843A1690843E1690843216ABE
:100D600008430543606A042803D1D4E90B01084312
:100D70000543206805602068456925F00705606A1D
:100D80000543606A04280DD1A06A0543E06A48B1B2
:100D90002046FFF753FC28B140206065012084F80D
:100DA0003500A6E7206845612046FFF72DFC064682
:100DB00094F85C103F208840B060002060650120FE
:100DC00084F83500002094E73F8010F02DE9F047CB
:100DD00004460D4616461F464FF00008D4F85890BA
:100DE00000BF94F83400012802D10220BDE8F0874A
:100DF000012084F8340000BF94F83500012825D183
:100E0000022084F83500002060653B4632462946C2
:100E10002046FFF768FC94F85C103F208840C9F832
:100E200008002068006840F0160021680860206C07
:100E300028B12068006840F0080021680860206838
:100E4000006840F001002168086006E000BF002053
:100E500084F8340000BF4FF002084046C6E70000A7
:100E600070B5044600F0E0F906462546681C10B14E
:100E700004480078054400BF00F0D6F9801BA84262
:100E8000FAD370BD080000202DE9F04104460E465B
:100E90000127002500BF2548007E012802D102203D
:100EA000BDE8F08101202149087600BF4CF25030A6
:100EB000FFF75AFD0746002F31D1401E30602068F1
:100EC00001280FD1207C6168FFF792FC4CF2503072
:100ED000FFF74AFD07461648006820F00400144951
:100EE00008601AE0A56812E0217C2846FFF716FC8E
:100EF0004CF25030FFF738FD07460D48006820F0EF
:100F0000FA000B4908600FB1356005E06D1CD4E9AB
:100F100002100844A842E7D800BFFFF72DFC00BF2D
:100F200000200249087600BF3846B9E728060020AD
:100F3000103C02400348006840F00040014908604E
:100F400000207047103C02402DE9F04106460F4654
:100F500014461D464FF0010800BF1F48007E0128BF
:100F600002D10220BDE8F08101201B49087600BFB4
:100F70004CF25030FFF7F8FC8046B8F1000F23D157
:100F800026B9E1B23846FFF74BFC12E0012E04D13E
:100F9000A1B23846FFF774FC0BE0022E04D12146C3
:100FA0003846FFF781FC04E022462B463846FFF71F
:100FB00049FC4CF25030FFF7D7FC804607480068E8
:100FC00020F001000549086000BF002002490876B2
:100FD00000BF4046C6E7000028060020103C024043
:100FE00000200949096801F0004159B10749064A42
:100FF0000C3A1160064911600349096801F000418B
:1010000001B1012070470000103C024023016745F8
:10101000AB89EFCDF8B502460B4600250024002031
:101020000021D6E0012606FA01F51E6806EA05044D
:10103000AC4274D11E7906F00306012E04D01E794D
:1010400006F00306022E13D190684F000326BE401F
:10105000B0434F00DE68BE403043906050680126C8
:101060008E40B0431E79C6F300168E403043506068
:101070001E7906F00306032E09D0D0684F00032620
:10108000BE40B0434F009E68BE403043D0601E79E2
:1010900006F00306022E13D1CF0802F1200656F8FF
:1010A00027004E07F70E0F26BE40B0434F07FF0E36
:1010B0001E69BE403043CF0802F1200646F82700E3
:1010C00010684F000326BE40B0431E7906F00306A9
:1010D0004F00BE40304310605E6806F44036002E7C
:1010E00076D000BF002600963C4E366846F4804617
:1010F0003A4F3E603E46366806F48046009600BF92
:1011000000BF374E8F0856F827008E07370F0F267F
:10111000BE40B043334EB24202D1002624E057E035
:10112000314EB24201D101261EE0304EB24201D111
:10113000022619E02E4EB24201D1032614E02D4EB4
:10114000B24201D104260FE02B4EB24201D1052656
:101150000AE02A4EB24201D1062605E0284EB242EC
:1011600001D1072600E008268F073F0FBE4030431D
:101170001B4E8F0846F82700224E3068A0435E6859
:1011800006F4801606B120431E4E3060361D3068CE
:10119000A0435E6806F4001606B12043194E361DC2
:1011A0003060184E361F3068A0435E6806F4003683
:1011B00006B12043134E361F3060361F3068A043FF
:1011C0005E6806F4803606B120430E4E083E30605D
:1011D000491C1029FFF426AFF8BD00004438024036
:1011E00008380140000002400004024000080240AC
:1011F000000C02400010024000140240001802409F
:10120000001C0240083C014010B5426921EA02037B
:1012100002EA010443EA0443836110BD0AB181611B
:1012200001E00B04836170470148006870470000CB
:101230000000002003480068034909780844014978
:1012400008607047000000200800002010B50D481D
:10125000006840F400700B4908600846006840F4DC
:10126000806008600846006840F4807008600320D1
:1012700000F0A6F8032000F007F800F02BF800209B
:1012800010BD0000003C024070B504460E480078D6
:101290004FF47A71B1FBF0F00C490968B1FBF0F53D
:1012A000284600F02FFC08B1012070BD102C07D299
:1012B00000222146501E00F045F80548046001E078
:1012C0000120F2E70020F0E7080000200C000020D9
:1012D0000400002008B500BF0020009010480068FE
:1012E00040F480400E4908600846006800F48040E1
:1012F000009000BF00BF00BF00200090081F0068E2
:1013000040F08050091F08600846006800F08050D7
:10131000009000BF00BF052000F052F808BD00009B
:101320004438024001460846002809DB00F01F034C
:1013300001229A4043099B0003F1E023C3F80021F6
:1013400000BF70472DE9F05F80460D461646002726
:1013500001F062FE074639462A46334601F007008F
:10136000C0F1070ABAF1040F02D94FF0040A01E0F4
:10137000C0F1070AD14600F1040ABAF1070F02D200
:101380004FF0000A01E0A0F1030AD4464FF0010A31
:101390000AFA09FAAAF1010A0AEA020A0AFA0CFA96
:1013A0004FF0010B0BFA0CFBABF1010B0BEA030B3B
:1013B0004AEA0B042146404601F036FEBDE8F09FA4
:1013C00000BF00F00702064B19684FF6FF031940F3
:1013D000044B0B4343EA0221014B196000BF7047E5
:1013E0000CED00E00000FA0570B504460D460CB99E
:1013F000012070BD5848006800F00700A84209D2DB
:1014000055490D700846006800F00700A84201D059
:101410000120EEE7207800F0020002281DD120789C
:1014200000F00400042805D14C48006840F4E05066
:101430004A490860207800F00800082805D147488C
:10144000006840F46040454908604448006820F066
:10145000F000A168084341490860207800F00100CD
:10146000A8B36068012807D13C4808380068C0F379
:101470004040B8B90120BCE76068022802D060682B
:10148000032807D1354808380068C0F3406048B9E0
:101490000120AEE7314808380068C0F3400008B9C1
:1014A0000120A6E72D48006820F00300616808438A
:1014B0002A490860FFF7B8FE064609E0FFF7B4FEC8
:1014C000801B41F28831884202D9032091E707E06E
:1014D0002248006800F00C006168B0EB810FEDD18C
:1014E0001D48006800F00700A84209D91A490D708C
:1014F0000846006800F00700A84201D0012078E704
:10150000207800F00400042807D11448006820F473
:10151000E050E168084311490860207800F00800B5
:10152000082808D10D48006820F46040216940EA8D
:10153000C1000A49086000F03FF808490968C1F392
:101540000311074A515CC840064908600648006814
:10155000FFF79AFE00204CE7003C024008380240AA
:101560000A3900080C00002004000020014800682F
:10157000704700000C00002000B5FFF7F7FF04499A
:101580000968C1F38221034A515CC84000BD0000D4
:10159000083802401A39000800B5FFF7E7FF044990
:1015A0000968C1F34231034A515CC84000BD0000E4
:1015B000083802401A3900082DE9F04700240025B8
:1015C0000026A1462548006800F00C0020B1042840
:1015D00005D008283AD105E0DFF8849039E0DFF83B
:1015E000849036E01D48001F006800F03F041B484F
:1015F000001F006800F4800078B11A481749091FDD
:101600000968C1F38811A0FB01700146224600233E
:101610003846FEF749FE05460EE011480F49091FFE
:101620000968C1F38811A0FB01700146224600231E
:101630003846FEF739FE05460848001F0068C0F32B
:101640000140401C4600B5FBF6F902E0DFF81090BF
:1016500000BF00BF4846BDE8F087000008380240E0
:101660000024F40000127A00F8B504460CB90120F9
:10167000F8BD207800F00100002874D0F948006817
:1016800000F00C0004280DD0F648006800F00C00B3
:10169000082813D1F348001F006800F48000B0F55B
:1016A000800F0BD1EF4808380068C0F34040002895
:1016B00059D06068002856D10120D9E700BF606882
:1016C000B0F5803F08D1E7480838006840F4803022
:1016D000E449083908601EE06068B0F5A02F0DD11C
:1016E000E0480838006840F48020DE490839086086
:1016F0000846006840F4803008600CE0D94808389B
:10170000006820F48030D74908390860084600682E
:1017100020F48020086000BF606890B1FFF784FD6E
:10172000054606E0FFF780FD401B642801D9032031
:101730009EE7CC4808380068C0F340400028F1D04C
:1017400011E0FFF771FD054606E0FFF76DFD401B58
:10175000642801D903208BE7C24808380068C0F329
:1017600040400028F1D1207800F0020002285FD12B
:10177000BC48006800F00C0058B1BA48006800F09E
:101780000C0008281CD1B748001F006800F4800036
:10179000B0B9B44808380068C0F3400020B1E06830
:1017A000012801D0012063E7AE480838006820F026
:1017B000F800216940EAC100AA490839086037E009
:1017C000E06800B30120A8490860FFF72DFD054639
:1017D00006E0FFF729FD401B022801D9032047E757
:1017E000A04808380068C0F340000028F1D09D48A8
:1017F0000838006820F0F800216940EAC1009949E2
:101800000839086014E0002097490860FFF70CFDD4
:10181000054606E0FFF708FD401B022801D903201A
:1018200026E7904808380068C0F340000028F1D14E
:10183000207800F0080008282CD16069A8B10120A8
:101840008A490860FFF7F0FC054606E0FFF7ECFC6C
:10185000401B022801D903200AE782486C30006847
:10186000C0F340000028F1D014E000207F49086058
:10187000FFF7DAFC054606E0FFF7D6FC401B02281E
:1018800001D90320F4E677486C300068C0F34000CB
:101890000028F1D1207800F00400042870D100273E
:1018A00070483830006800F0805090B900BF0020C8
:1018B00000906C483830006840F0805069493831F9
:1018C00008600846006800F08050009000BF00BF2C
:1018D00001276748006800F48070B0B96448006868
:1018E00040F4807062490860FFF79EFC054606E000
:1018F000FFF79AFC401B022801D90320B8E65C4898
:10190000006800F480700028F2D000BFA0680128B1
:1019100008D154486830006840F0010051496831EE
:1019200008601DE0A06805280DD14E4868300068A9
:1019300040F004004B49683108600846006840F0F8
:10194000010008600CE047486830006820F00100A2
:101950004449683108600846006820F004000860C7
:1019600000BFA068A8B1FFF75FFC054609E0FFF7DC
:101970005BFC401B41F28831884202D9032077E6A4
:1019800026E0384868300068C0F340000028EED0F8
:1019900013E0FFF749FC054608E0FFF745FC401B54
:1019A00041F28831884201D9032061E62D48683030
:1019B0000068C0F340000028EFD1012F07D129486B
:1019C0003830006820F0805026493831086000BF68
:1019D000A069002845D02348006800F00C000828C2
:1019E0005DD0A069022845D100201F490866FFF795
:1019F0001BFC054606E0FFF717FC401B022801D937
:101A0000032035E6174808380068C0F34060002816
:101A1000F1D1D4E907010843616A40EA811101224A
:101A2000A06AC2EB500041EA00412C20005D41EA6F
:101A300000600C49091F086001200B490866FFF788
:101A4000F3FB054606E0FFF7EFFB401B022801D938
:101A500003200DE6034808380068C0F34060002802
:101A6000F1D049E00838024000004742800E47426A
:101A700000700040002021490866FFF7D5FB0546AD
:101A800006E0FFF7D1FB401B022801D90320EFE558
:101A90001B480068C0F340600028F2D12CE0A06928
:101AA000012800D1E4E51648001D0668A069012858
:101AB00020D006F48001E06981421BD106F03F018D
:101AC000206A814216D147F6C0703040616AB0EB9F
:101AD000811F0FD106F440310122A06AC2EB5000F1
:101AE000B1EB004F06D106F070612C20005DB1EB28
:101AF000006F01D00120BBE50020B9E5000047429E
:101B00000038024070B504462546681EB0F1807F5B
:101B100001D301200FE0681E4FF0E02148610F2142
:101B20004FF0FF3001F080FA00204FF0E021886193
:101B300007200861002070BDF8B504460E46174620
:101B400094F83E00202836D106B10FB90120F8BD27
:101B500000BF94F83C00012801D10220F7E70120E2
:101B600084F83C0000BF20633A463146204601F02D
:101B7000A9F90546EDB9206B012819D100BF002055
:101B8000009020680068009020684068009000BFC6
:101B900000BF00BF00BF21680C3151E8001F41F0B9
:101BA000100021680C3141E80002002AF3D100E066
:101BB00001252846CBE70220C9E7000070B504469E
:101BC0000D460C492068884203D10B4801F0E8FC1F
:101BD0000EE00A492068884203D1094801F0E0FC80
:101BE00006E008492068884202D1074801F0D8FC85
:101BF00070BD000000100140F801002000440040CA
:101C000048020020004C00409802002070B50446B5
:101C1000002520684069C0F3C01594F83D002128D4
:101C200017D1B5B100BF00BF2168143151E8001FC2
:101C300021F080002168143141E80002002AF3D12C
:101C400000BF606B10B1606BFEF7C0FE204600F075
:101C500094FF20684069C0F3801594F83E00222864
:101C600017D1B5B100BF00BF2168143151E8001F82
:101C700021F040002168143141E80002002AF3D12C
:101C800000BFA06B10B1A06BFEF7A0FE204600F0D5
:101C90002EFF002070BD000038B5044600252B49FA
:101CA0002068884201D12A4D0AE02A4920688842EA
:101CB00001D1294D04E029492068884200D1284DEE
:101CC000206C00F0020050B100BF0020009020689E
:101CD0000068009020684068009000BF00BF206C42
:101CE00000F0040050B100BF0020009020680068A0
:101CF000009020684068009000BF00BF2068006826
:101D0000C0F3C00050B100BF002000902068006800
:101D1000009020684068009000BF00BF2068006805
:101D2000C0F3400050B100BF002000902068006860
:101D3000009020684068009000BF00BF25B1EA8B8A
:101D4000A9696868FFF7F8FE38BD0000001001407F
:101D5000F80100200044004048020020004C0040F0
:101D6000980200202DE9F84F044620680568206895
:101D7000C668206847694FF00009CA4605F00F0998
:101D8000B9F1000F0AD105F0200038B106F02000AB
:101D900020B1204600F004FFBDE8F88FB9F1000F34
:101DA0007CD007F0010018B906F49070002875D0B7
:101DB00005F0010030B106F4807018B1206C40F0DD
:101DC0000100206405F0040030B107F0010018B1F3
:101DD000206C40F00200206405F0020030B107F0F2
:101DE000010018B1206C40F00400206405F00800E8
:101DF00048B106F0200010B907F0010018B1206CBE
:101E000040F008002064206C002846D005F0200037
:101E100028B106F0200010B1204600F0C1FE206875
:101E20004069C0F3801A206C00F0080010B9BAF1C4
:101E3000000F2DD0204600F05AFE2068406900F0C7
:101E40004000402820D100BF00BF2168143151E874
:101E5000001F21F040002168143141E80002002AEF
:101E6000F3D100BFA06B50B17548A16B0865A06BA2
:101E7000FEF702FE88B1A06B016D88470DE0204699
:101E8000FFF70AFF09E009E02046FFF705FF04E03D
:101E90002046FFF701FF002020647DE7206B01282A
:101EA00076D105F01000002872D006F0100000284E
:101EB000FAD000BF002000902068006800902068E1
:101EC0004068009000BF00BF2068406900F04000FB
:101ED00040285ED1A06B006840681FFA80F8B8F116
:101EE000000F54D0A08D404551DDA4F82E80A06B8A
:101EF000C069B0F5807F43D000BF00BF21680C31BE
:101F000051E8001F21F4807021680C3141E8000283
:101F1000002AF3D100BF00BF00BF2168143151E88F
:101F2000001F21F001002168143141E80002002A5D
:101F3000F3D100BF00BF00BF2168143151E8001F7A
:101F400021F040002168143141E80002002AF3D159
:101F500000BF202084F83E000020206300BF00BFA7
:101F600021680C3151E8001F21F0100021680C316C
:101F700041E80002002AF3D100BFA06BFEF726FD66
:101F8000A08DE28D801A81B22046FFF717FE03E78D
:101F900040E0A08DE18D401A1FFA80F8E08DC0B3BB
:101FA000B8F1000F35D000BF00BF21680C3151E8F7
:101FB000001F21F4907021680C3141E80002002AD2
:101FC000F3D100BF00BF00BF2168143151E8001FEA
:101FD00021F001002168143141E80002002AF3D108
:101FE00000BF202084F83E000020206300BF00BF17
:101FF00021680C3151E8001F21F0100021680C31DC
:1020000041E80002002AF3D100BF41462046FFF715
:10201000D5FDC1E605F0800030B106F0800018B1B2
:10202000204600F0B7FFB7E605F0400030B106F0FB
:10203000400018B1204600F090FDADE600BFABE6D1
:102040005529000810B504460CB9012010BDA0693F
:1020500000B100E000BF94F83D0028B9002084F8EA
:102060003C00204600F028F8242084F83D00206839
:10207000C06820F400502168C860204600F00CFEC3
:102080002068006920F49040216808612068406958
:1020900020F02A00216848612068C06840F40050A0
:1020A0002168C86000202064202084F83D0084F866
:1020B0003E000020CAE7000010B586B00446142197
:1020C00001A8FEF7D9F9C149206888427AD100BF3A
:1020D00000200090BE48006840F40020BC49086021
:1020E0000846006800F40020009000BF00BF00BF59
:1020F00000200090B6481038006840F00100B44954
:10210000103908600846006800F00100009000BF28
:1021100000BF0320019002200290002003900320C2
:1021200004900820059001A9AA48FEF773FFAA4869
:10213000AA490860400548600021A8488160C16044
:102140004FF480610161002141618161C1614FF4FF
:102150004031016200214162FEF7C2FD08B1FEF785
:10216000D9FA00BF9D48A063846300BF9A4830300D
:102170009B4908604FF000604860402198488160AA
:102180000021C1604FF480610161002141618161E2
:10219000C1614FF40031016200214162FEF7A0FDF0
:1021A00008B1FEF7B7FA00BF8D486063846300BFD3
:1021B000002201213420FFF7C5F83420FFF7B2F8E0
:1021C00002E1FFE78749206888427ED100BF0020F6
:1021D00000907F48001D006840F010007C49091DF8
:1021E00008600846006800F01000009000BF00BFC3
:1021F00000BF0020009076481038006840F00100D1
:102200007349103908600846006800F0010000902A
:1022100000BF00BF4FF4C060019002200290002078
:102220000390032004900720059001A96948FEF758
:10223000F1FE6D486D4908604FF000604860002174
:102240006A488160C1604FF4806101610021416191
:102250008161C1614FF48031016200214162FEF76A
:102260003FFD08B1FEF756FA00BF6048A0638463E3
:1022700000BF5D4878305E4908604FF000604860FC
:1022800040215B4881600021C1604FF480610161A1
:10229000002141618161C1614FF4803101620021FF
:1022A0004162FEF71DFD08B1FEF734FA00BF504849
:1022B0006063846300BF002201212520FFF742F8FC
:1022C0002520FFF72FF87FE0FFE74A492068884282
:1022D0007AD100BF002000903D48006840F40030F3
:1022E0003B4908600846006800F40030009000BFD9
:1022F00000BF00BF0020009035481038006840F053
:1023000008003349103908600846006800F00800EA
:10231000009000BF00BF60200190022002900020CA
:102320000390032004900720059001A93248FEF78E
:1023300071FE29484830314908604FF0006048601C
:1023400000212E488160C1604FF48061016100214D
:1023500041618161C1614FF44031016200214162FC
:10236000FEF7BEFC08B1FEF7D5F900BF2348A06315
:10237000846300BF18486030214908604FF0006056
:10238000486040211E4881600021C1604FF4806197
:102390000161002141618161C1614FF4003101623D
:1023A00000214162FEF79CFC08B1FEF7B3F900BFC3
:1023B00013486063846300BF002201212620FEF7DA
:1023C000C1FF2620FEF7AEFF06B010BD004C004056
:1023D000403802400000024040600240E803002014
:1023E000480400200010014040640240A80400207E
:1023F0000805002000440040000C02406805002051
:10240000C805002070477047F7B50446154694F894
:102410003D00202846D1019800B10DB90120FEBD34
:1024200000BF94F83C00012801D10220F7E7012009
:1024300084F83C0000BF01982062A584E584002058
:102440002064212084F83D001748616BC863174859
:10245000616B08641648616BC8640020616B086595
:1024600001AE23681A1D31682B46606BFEF7AEFC87
:102470006FF040002168086000BF002084F83C0035
:1024800000BF00BF00BF2168143151E8001F41F0B8
:1024900080002168143141E80002002AF3D100BF16
:1024A0000020BCE70220BAE7892A0008E12A0008D8
:1024B0006929000810B504460B492068884203D1F9
:1024C0000A4801F007F90EE009492068884203D163
:1024D000084801F0FFF806E007492068884202D169
:1024E000044801F0F7F810BD00100140F801002089
:1024F0000044004048020020004C0040704700BFEC
:10250000FEE7000008B500BF0020009026480068E4
:1025100040F40010244908600846006800F40010E8
:10252000009000BF00BF00BF002000900846006878
:1025300040F4800008600846006800F480000090C5
:1025400000BF00BF002211460D20FEF7FBFE0D204C
:10255000FEF7E8FE002211460F20FEF7F3FE0F20E3
:10256000FEF7E0FE002211461020FEF7EBFE1020E1
:10257000FEF7D8FE002211461120FEF7E3FE1120DF
:10258000FEF7D0FE002211463A20FEF7DBFE3A208D
:10259000FEF7C8FE002211464620FEF7D3FE462075
:1025A000FEF7C0FE08BD00003038024000B587B01D
:1025B000142102A8FDF760FF00BF002001906E48C3
:1025C000006840F010006C4908600846006800F0A0
:1025D0001000019000BF00BF00BF0020019008461E
:1025E000006840F0800008600846006800F0800045
:1025F000019000BF00BF00BF0020019008460068A6
:1026000040F0010008600846006800F001000190F9
:1026100000BF00BF00BF002001900846006840F0E6
:10262000020008600846006800F00200019000BF48
:1026300000BF00BF002001900846006840F008007D
:1026400008600846006800F00800019000BF00BF65
:1026500000BF002001900846006840F004000860B8
:102660000846006800F00400019000BF00BF00228F
:102670007F214248FEF7D2FD012204214048FEF7A7
:10268000CDFD01224FF4E0613C48FEF7C7FD012279
:102690004FF470413B48FEF7C1FD01224FF47F41EA
:1026A0003948FEF7BBFD01224FF470713748FEF741
:1026B000B5FD002210213448FEF7B0FD00224FF492
:1026C00040713048FEF7AAFD6F2002900120039070
:1026D000002004900320059002A92848FEF79AFCE8
:1026E0004FF4E260029001200390002004900590D6
:1026F00002A92248FEF78EFC0420029001200390DC
:10270000002004900320059002A91D48FEF782FCDA
:102710004FF4704002900120039000200490059037
:1027200002A91848FEF776FC4FF6107002900120BF
:10273000039000200490059002A91348FEF76AFC5C
:102740004FF47070029001200390002004900590D7
:1027500002A90E48FEF75EFC4FF440700290012083
:102760000390002004900320059002A90548FEF77D
:1027700051FC07B000BD000030380240001002409C
:102780000000024000040240000C02400008024029
:1027900010B50B480B4908604FF4E1304860002148
:1027A00008488160C16001610C21416100218161A3
:1027B000C161FFF747FC08B1FDF7ACFF10BD000099
:1027C000004C00401C03002010B50B480B4908606A
:1027D0004FF4E1304860002108488160C160016128
:1027E0000C21416100218161C161FFF72BFC08B11F
:1027F000FDF790FF10BD00000010014060030020B5
:1028000010B50B480B4908604FF416504860002182
:1028100008488160C16001610C2141610021816132
:10282000C161FFF70FFC08B1FDF774FF10BD000098
:1028300000440040A403002000BFFEE700BFFEE705
:102840007047704710B5094841690120884708481A
:102850000121426C904707480121426C904706488D
:102860000121426C9047FEF7E5FC10BD8C00002072
:10287000F8010020480200209802002000B593B023
:10288000302107A8FDF7F8FD142102A8FDF7F4FD9B
:1028900000BF002001902448006840F08050224989
:1028A00008600846006800F08050019000BF00BF3B
:1028B00000BF002001901D48006840F480401B4983
:1028C00008600846006800F48040019000BF00BF27
:1028D000012007900004089002200D9041050E9100
:1028E00004210F91A821109102211191042112912C
:1028F00007A8FEF7B9FE08B1FDF70CFF0F20029004
:1029000002200390002004904FF4A05005904FF453
:1029100080500690052102A8FEF766FD08B1FDF77C
:10292000F9FE13B000BD00004038024000700040C6
:102930000348006840F470000149086070470000D7
:1029400088ED00E010B50248FFF70CFA10BD00005A
:102950001C03002070B50546AC6B0020E085E084C8
:102960002046FFF799F970BD70B506460025B46B97
:1029700020684069C0F3C01594F83D00212805D1B6
:1029800025B10020E084204600F0F7F82068406977
:10299000C0F3801594F83E00222805D125B100200F
:1029A000E085204600F0A3F8206C40F01000206481
:1029B0002046FFF771F970BD70B50546AC6B28680D
:1029C000006800F48070002842D1E08500BF00BF9D
:1029D00021680C3151E8001F21F4807021680C310E
:1029E00041E80002002AF3D100BF00BF00BF216808
:1029F000143151E8001F21F001002168143141E831
:102A00000002002AF3D100BF00BF00BF21681431CB
:102A100051E8001F21F040002168143141E8000214
:102A2000002AF3D100BF202084F83E00206B01284B
:102A30000ED100BF00BF21680C3151E8001F21F00A
:102A4000100021680C3141E80002002AF3D100BFD8
:102A5000206B012804D1A18D2046FFF7AFF802E0DA
:102A60002046FFF7CFFC70BD70B50546AC6B206B00
:102A7000012805D1A08D41082046FFF79FF802E00C
:102A80002046FFF7C0FC70BD70B50546AC6B2868EA
:102A9000006800F48070F8B90020E08400BF00BF37
:102AA0002168143151E8001F21F0800021681431A1
:102AB00041E80002002AF3D100BF00BF00BF216837
:102AC0000C3151E8001F41F0400021680C3141E811
:102AD0000002002AF3D102E02046FFF7EBFC70BDB4
:102AE00070B50446A56B2846FFF708FD70BD00BF12
:102AF00000BF02680C3252E8002F22F49071026885
:102B00000C3242E80013002BF3D100BF00BF00BF1E
:102B10000268143252E8002F22F0010102681432D8
:102B200042E80013002BF3D100BF016B01290ED145
:102B300000BF00BF02680C3252E8002F22F01001E3
:102B400002680C3242E80013002BF3D100BF2021B1
:102B500080F83E1000210163704710B504462068DC
:102B6000C06820F040002168C860202084F83D0043
:102B70002046FFF79FFC002010BD00BF00BF026889
:102B80000C3252E8002F22F0C00102680C3242E8F9
:102B90000013002BF3D100BF202180F83D107047B7
:102BA000F8B5044694F83E00222873D1A068B0F529
:102BB000805F0CD1206950B90025A66A2068406862
:102BC000C0F308003080A06A801CA06215E0A56AEE
:102BD0000026A068B0F5805F03D0A06828B92069FE
:102BE00018B920684068287004E02068406800F048
:102BF0007F002870A06A401CA062E08D401E80B259
:102C0000E085002844D12068C06820F020002168B9
:102C1000C8602068C06820F480702168C86020689F
:102C2000406920F0010021684861202084F83E00BE
:102C3000206B012826D10020206300BF00BF21683F
:102C40000C3151E8001F21F0100021680C3141E8DF
:102C50000002002AF3D100BF2068006800F01000D5
:102C600010280AD100BF0020009020680068009062
:102C700020684068009000BF00BFA18D2046FEF78D
:102C80009DFF02E02046FFF7BDFB0020F8BD01E0FC
:102C90000020FBE70220F9E72DE9F84F0446206801
:102CA000006920F44050E168084321680861216907
:102CB000A068084361690843E169084300902068FF
:102CC000C06849F20C618843009908432168C860D4
:102CD0002068406920F44070A16908432168486178
:102CE00076492068884203D075492068884203D11C
:102CF000FEF752FC814602E0FEF73EFC8146E069A9
:102D0000B0F5004F6CD102206168A0FB0150034672
:102D10001920A9FB007001462A463846FDF7C4FA7F
:102D20006421B0FBF1F04FEA001A02206168A0FBB9
:102D300001510B461920A9FB00712A463846FDF7C0
:102D4000B3FA834602206168A0FB015003461920B4
:102D5000A9FB00712A463846FDF7A6FA6421B0FBAC
:102D6000F1F000EBC00101EB0010ABEB8000322171
:102D700001EBC0006421B0FBF1F000F0F8000AEBB9
:102D8000400A02206168A0FB015003461920A9FBFC
:102D9000007001462A463846FDF786FA834602202F
:102DA0006168A0FB015003461920A9FB00712A4667
:102DB0003846FDF779FA6421B0FBF1F000EBC00171
:102DC00001EB0010ABEB8000322101EBC00064216D
:102DD000B0FBF1F000F007005044216888606AE021
:102DE00004206168A0FB015003461920A9FB007074
:102DF00001462A463846FDF757FA824604206168A4
:102E0000A0FB015003461920A9FB007001462A4689
:102E10003846FDF749FA6421B0FBF1F000EBC00140
:102E200001EB0010AAEB8000322101EB00106421BD
:102E3000B0FBF1F000F0F00A04206168A0FB017023
:102E400003461920A9FB00513A462846FDF72CFA03
:102E50006421B0FBF1F00AEB001A04206168A0FBCA
:102E600001510B461920A9FB00712A463846FDF78F
:102E70001BFA834604206168A0FB01500346192019
:102E8000A9FB007001462A463846FDF70DFA642179
:102E9000B0FBF1F000EBC00101EB0010ABEB8000E8
:102EA000322101EB00106421B0FBF1F000F00F00C3
:102EB000504421688860BDE8F88F00000010014090
:102EC0000014014077B581B0044615460298A0620F
:102ED000A58500202064222084F83E002A48A16BAA
:102EE000C8632A48A16B08642948A16BC864002004
:102EF000A16B086502AE32682368191D2B46A06BD2
:102F0000FDF764FF00BF002000902068006800907B
:102F100020684068009000BF00BF00BF002084F818
:102F20003C0000BF206970B100BF00BF21680C31B8
:102F300051E8001F41F4807021680C3141E8000223
:102F4000002AF3D100BF00BF00BF2168143151E84F
:102F5000001F41F001002168143141E80002002AFD
:102F6000F3D100BF00BF00BF2168143151E8001F3A
:102F700041F040002168143141E80002002AF3D1F9
:102F800000BF002004B070BDB9290008692A0008FC
:102F900069290008014691F83D00212828D1886858
:102FA000B0F5805F0BD1086948B90A6A1088C0F390
:102FB00008000B685860086A801C086205E00B6A0C
:102FC000581C086218780B685860C88C401E80B284
:102FD000C88458B90868C06820F080000B68D860C1
:102FE0000868C06840F040000B68D8600020704757
:102FF0000220FCE710B50248FEF7B4FE10BD000049
:103000006003002010B50248FEF7ACFE10BD0000C2
:10301000A403002000BFFEE702480068C0F30220BE
:10302000704700000CED00E010B5002804DB0A0733
:10303000130E054A135406E00A07140E034A00F063
:103040000F031B1FD45410BD00E400E018ED00E096
:1030500010B50D49086A80470C48416B88470C48F9
:10306000416B88470B48416B88470B49086880478C
:103070000A480B49C268082090470A4948688047B7
:1030800009490868804710BD7C010020F801002034
:103090004802002098020020700100208C000020CF
:1030A0002C00002010030020A800002010B50349C8
:1030B0000869804700F00EFC10BD00008C00002065
:1030C000034A12689080024A1268916070470000BB
:1030D000A400002010B51A480068806800B910BD2F
:1030E000002425E016480068806804EB440110F8CD
:1030F0002100D0B1002012490968896804EB44021C
:1031000001F822000E480068806804EB440100EBDF
:103110008100806800B909E009490968896804EB01
:10312000440201EB82018868804700BF601C84B2C2
:10313000034800688088A042D4DC00BFCFE70000CD
:10314000A400002010B501462F4A12681288521CB4
:103150002D4B1B681A802C4A12681288B2F57A7FB0
:1031600006DB294A12685288521C274B1B685A807A
:10317000254A1268926802B910BD00203CE0224A3C
:103180001268926800EB400302EB830252888AB314
:103190001D4A1268926800EB400302EB83025288DA
:1031A000521E194B1B689B6800EB400403EB840321
:1031B0005A80154A1268926800EB400302EB8302C2
:1031C0005288BAB90122104B1B689B6800EB40047F
:1031D00003F824200C4A1268926800EB400302EBCB
:1031E00083029288084B1B689B6800EB400403EB4A
:1031F00084035A80421C90B2034A12689288824229
:10320000BDDC00BFB8E70000A40000200148007842
:10321000704700006C01002010B5002007490870BD
:10322000002210210648FDF7F9FF00221021054871
:10323000FDF7F4FF002000F007F810BD6C0100203E
:1032400000100240000C02402DE9F04180460025AC
:10325000102D01DBBDE8F0812C4805702C48465D3F
:103260002C48475D002431E046FA04F000F00100EC
:1032700048B1294A32F81410284A52F82400012291
:10328000FDF7CCFF08E0244A32F81410234A52F824
:1032900024000022FDF7C2FF47FA04F000F001000D
:1032A00048B11F4A32F814101E4A52F82400012275
:1032B000FDF7B4FF08E01A4A32F81410194A52F820
:1032C00024000022FDF7AAFF601CC4B2042CCBDB53
:1032D000002416E0AC4209D1134A32F81410134A04
:1032E00052F824000022FDF799FF08E00E4A32F858
:1032F00014100E4A52F824000122FDF78FFF601CC3
:10330000C4B2102CE6DB00BFA4E700006C01002073
:103310004C0100205C010020CC000020BC000020FB
:10332000E4000020D40000202C010020EC0000204C
:1033300010B586B00446002001900B2003900120B8
:1033400004900220059000200090694601A8FDF736
:103350009BFD06B010BD000010B5064948688047C7
:1033600010220549054800F055F802494868804791
:1033700010BD0000B00000208C01002000000E08ED
:1033800070B510220E49A1F11000FDF704F8A8B1A4
:103390000C494868804772B6102209490A4800F073
:1033A0005DF804462CB906481038054610352ECD78
:1033B0002EC062B603494868804700BF70BD000058
:1033C0008C010020B000002000000E0810B5FFF7AF
:1033D000D7FF10BD10B5FFF7BFFF0C480068808B0A
:1033E000B0F57A7F03DD282108480068818307480B
:1033F0000068C08B102803DD102104480068C183D9
:103400000348044610341ECC1EC010BDAC01002081
:103410007C0100202DE9F84103460C4621461D465B
:10342000960802F00307002005E055F820C0C1F817
:1034300000C0091D401CB042F7D36FB155F82600FB
:103440000090EC46002004E01CF8008001F80080A9
:10345000401CB842F8D300BFBDE8F8812DE9FC5FFD
:1034600007468846154600244646A808019005F000
:103470000309BA46FDF7B4FD3846FFF759FF044685
:1034800024B1FDF757FD2046BDE8FC9F4FF0000B2F
:103490000FE0D6F800C06246002351460220FDF737
:1034A00053FD044604B107E00AF1040A361D0BF18E
:1034B000010B01988345ECD300BFB4B9B9F1000FFB
:1034C00013D04FF0FF300090EB46002003E0315C5A
:1034D0000BF80010401C4845F9D300235146022048
:1034E000009AFDF731FD044600BFFDF723FD20469D
:1034F000CAE770477047000010B5002409E0322089
:1035000000F0EBF84FF480710348FDF77DFE601C7E
:10351000C4B2142CF3DB10BD0010024010B54FF400
:1035200080710248FDF770FE10BD000000100240DF
:103530002DE9F0410446884617460020A074A08B70
:10354000B84200DAA78B3A4641466069FCF74FFF64
:103550003A4661696068FEF757FFFDF765FE05466C
:1035600008E0FDF761FE0646701BC82802D901205D
:10357000A07402E0A07C0028F3D000BFBDE8F08179
:1035800010B5044660680068C06840F010006168CB
:103590000968C860E28BA1696068FEF7CDFA10BDCA
:1035A00070B504466068FEF731FBE08BE16809689E
:1035B0004968401A86B206B970BD002506E0A269C6
:1035C0005119206800F04BF9681C85B2B542F6DB52
:1035D000204600F041F8E28BA1696068FEF7ACFA82
:1035E00000BFE9E770B50446A08C618C884227DAF9
:1035F000206880892084204600F034F8208CE18BFC
:1036000088421DDC208CD8B1208C40F6B83188422D
:1036100003D9206800F0D7F812E0002506E0094A37
:103620005119206800F0D7F8681C85B2208CA84298
:10363000F5DCA06C20B1218C22460248A36C98478F
:1036400070BD0000C06F002090F82620012A02D132
:10365000428C0A4442847047012180F826100021E0
:1036600041847047002180F8261041847047000093
:103670002DE9F04104460F4616461448844204D111
:10368000012204211248FDF7C9FDA08B96FBF0F042
:103690001FFA80F8002507E0A28B02FB0571204687
:1036A000FFF746FF681C85B24545F5DBA08B00FBA4
:1036B000156086B20EB9BDE8F081A08B00FB0571E4
:1036C00032462046FFF734FF00BFF4E7980200209F
:1036D0000000024001218174704710B50446204665
:1036E000FDF7BEFB10BD2DE9F04704460D4691469F
:1036F000052D01DABDE8F0872078AA2802D160788C
:10370000552800D0F6E7681E215CA81E205C41EA1F
:103710000028A81E81B2204600F037F80646301275
:1037200040EA062086B2464500D0E3E7A778032F9B
:1037300000D100BF00BFDDE701480249886470473F
:10374000E7360008F8010020FDF780FDFFF796F846
:10375000FEF72CFFFEF7D6FEFFF71AF8FFF734F856
:10376000FFF74EF8FFF774FC01E0FFF79FFCFCE762
:1037700070B503460C4603E014F8015B03F8015BE7
:10378000151EA2F10102F7D170BD30B502464FF609
:10379000FF7012E012F8014B6040002308E000F0D7
:1037A000010424B14AF2010484EA600000E0401000
:1037B0001C465D1CABB2082CF1DB0C1EA1F101050F
:1037C000A9B2E7D130BD00B9704700214161016164
:1037D000C16000BFF8E770B504460D460CB9002083
:1037E00070BDE06808B90020FAE745B1D4E90006E9
:1037F000236903FB060132462846FFF7B9FF20691B
:10380000401CA16890FBF1F201FB12002061E0680E
:10381000401EE0600120E3E770B504460D460CB998
:10382000002070BDD4E90210884201D10020F8E7E1
:1038300045B1D4E90016636903FB061032462946F8
:10384000FFF796FF6069401CA16890FBF1F201FB55
:1038500012006061E068401CE0600120E1E770B5A3
:1038600004460D460CB9002070BDD4E90210884210
:1038700004DA29462046FFF7CFFFF5E745B1D4E942
:103880000016636903FB061032462946FFF770FFF6
:103890006069401CA16890FBF1F201FB12006061BD
:1038A0002069401CA16890FBF1F201FB120020612D
:1038B0000120D9E770477047704770477047000094
:1038C00010B502494868804710BD0000A8000020DC
:1038D0007047000010B50548C16C88470448C16CAA
:1038E00088470448C16C884710BD0000F8010020DB
:1038F00048020020980200204FF04070E1EE100ACC
:1039000070470006101600061016000000000000A8
:10391000000001020304060708090000000001027C
:103920000304000056312E300000000031313532E2
:103930003030000031393230300000003537363059
:1039400030000000393630300000000034383030AC
:1039500000000000434F4D3100000000434F4D3246
:1039600000000000434F4D3300000000434F4D3432
:103970000000000094390008000000201C03000033
:10398000C40100081C3B00081C030020BC88000088
:103990002002000841321042011324F4132439009C
:1039A0000A120856302E3030312E303A012813D505
:1039B0003822081203320A3AB70C120732323AD1CF
:1039C0000C120B32643AB50C120D32C83ABB0C1211
:1039D000111AF43D3AC10C121323E8033AB90C1240
:1039E0001723D0073ABD0CA113C1301B08D504130F
:1039F000453123088C1420F93414081D351B08F5B3
:103A0000081AF3041AB01411AC100240041A40133F
:103A100012081A04D159144A04042A02B629051AB4
:103A20000810A9040A1D0C04594079041944128095
:103A300022402905197E396D29585910100E0D0E96
:103A40000F0C0B0A090807040302011B06051016D8
:103A500008090A0B0C1F010203040506E6211319CD
:103A6000321B0849041A0D04012013D5331B0881A9
:103A7000041A59041ACD04137C01142048061A2094
:103A8000CE11F3B80B0A1412180B14B81D181AB083
:103A90004C136003142008051C20A804BE19C7138A
:103AA000702914202835FC20B80B5E511381351481
:103AB0000871361B08D5041AA10C1A4908411AE5E9
:103AC0000C1AC8501AA4501AC8501A680429501366
:103AD000E0400C1020984C502B980220091C501AE2
:103AE000E0501A1C501A489C1AE80829501B5058DC
:103AF000B00A3464A01354391B085C041A64041A15
:103B00006C041A4C041A44041A34041A3C041A2C87
:0C3B100004811339371B081074000000FA
:040000050800018965
:00000001FF
